:0200000480007A
:100000009710000093800000171100001301810178
:1000100083A1000013D2110093D2F10013D3F10198
:1000200093D3010013D40101232031002322410086
:10003000232451002326610023287100232A8100F4
:1000400097100000938040FC17110000130101FF7E
:1000500003A40000935414001355F4009355F401C5
:10006000135604009356040123208100232291009B
:100070002324A1002326B1002328C100232AD10074
:1000800097100000938080F817110000130181FC85
:1000900083A6000013D7160093D7F60013D8F601F5
:1000A00093D8060013D906012320D1002322E100B2
:1000B0002324F1002326010123281101232A2101F1
:1000C000171600001306C6F497160000938606FA6A
:1000D0000329060093591900135AF900935AF9019C
:1000E000135B0900935B090123A0260123A23601BB
:1000F00023A4460123A6560123A8660123AA76015C
:1001000017160000130606F197160000938686F76F
:10011000832B060013DC1B0093DCFB0013DDFB01CB
:1001200093DD0B0013DE0B0123A0760123A28601D1
:1001300023A4960123A6A60123A8B60123AAC601DB
:10014000171D0000130D4DED971D0000938D0DF54B
:10015000032E0D00935E1E0013DF1E00935F1F0031
:1001600093D01F0013D110009351110023A0CD0193
:1001700023A2DD0123A4ED0123A6FD0123A81D0078
:1001800023AA2D0023AC3D0097100000938000E9C6
:1001900017110000130141F283A2000013D01200D6
:1001A0002320010097100000938080E717110000C2
:1001B0001301C1F083A2000013D01200935210006B
:1001C000232001002322510017150000130585E5A7
:1001D00097150000938505EF370610F01306C6F259
:1001E0006306B5028326C5002320D600832685003A
:1001F0002320D600832645002320D6008326050031
:100200002320D600130505016FF09FFD370510F080
:10021000130505F223200500000000000000000087
:0402200000000000DA
:101000000000000001000000FFFFFFFFFFFFFF7F67
:101010000000008010EFCDAB7856341298BADCFE99
:10102000FFFFFFFFFFFFFFFFFFFFFFFFFFFFFFFFD0
:10103000FFFFFFFFFFFFFFFFFFFFFFFFFFFFFFFFC0
:10104000FFFFFFFFFFFFFFFFFFFFFFFFFFFFFFFFB0
:10105000FFFFFFFFFFFFFFFFFFFFFFFFFFFFFFFFA0
:10106000FFFFFFFFFFFFFFFFFFFFFFFFFFFFFFFF90
:10107000FFFFFFFFFFFFFFFFFFFFFFFFFFFFFFFF80
:10108000FFFFFFFFFFFFFFFFFFFFFFFFFFFFFFFF70
:10109000FFFFFFFFFFFFFFFFFFFFFFFFFFFFFFFF60
:1010A000FFFFFFFFFFFFFFFFFFFFFFFFFFFFFFFF50
:1010B000FFFFFFFFFFFFFFFFFFFFFFFFFFFFFFFF40
:040000058000000077
:00000001FF
